:020000040000FA
:10000000000B6E006F00700071008907090A6A0218
:10001000AA02A9070D0A6B02AB0203040A032A0015
:100020002C000306AC0203040B032B002D00030677
:10003000AD020A028906200AEE010C02F001230A31
:10004000AE000C02B0000B02A9062A0AEF010D0255
:10005000F1010008AF000D02B1000008070EE20137
:10006000870883088608380A85088108840880087C
:100070006607850882083200080C34004605BD0971
:10008000B4091206450A4605460A4604470A480AC4
:10009000B4093203F402410A4604B409BD09500A06
:1000A000000833007500080C34002704070206001E
:1000B00007040702060026040604AE0926052705E4
:1000C00007020600BD09AB09BA09330303066A0A31
:1000D00006046C0A0605B502A809F402630AAB0916
:1000E000BA091506750A0605760A0604A809AB09B9
:1000F000BA090605A809AB09A80907050702060001
:100100000607800A270407020600260400082705C0
:10011000070206000705070206007300080C3400FA
:100120000606900AAB09A8093303AB09BD09060608
:100130009B0AF3049C0AF305A809F402940AAB098C
:10014000A809AB09A809270407020600260400082D
:100150002607A80A00082606AB0A0008190C280082
:100160000000E802B00A0008CF0C2800B00AFA0C20
:0E0170002800B00ABB0ABC0A0000000000080C
:10020000800C02003B0C27000600000C2600FF0CAF
:100210003600B70987091302AA0F4306120BF6022C
:10022000090B130B8709FF0C51098709AE098709D0
:100230001302AA0F4307160B8709EA0C5109870915
:10024000F40C510987092705070206000705070274
:1002500006000606290B87091302290087091302E5
:100260002A00870913022B00010909022E093B0904
:100270000E023B090F023B0910023B0911023B0928
:10028000230B4208590820084A084A0831084F0839
:0402900044084D08C9
:021FFE00E90FE9
:00000001FF
